:10000000B8C1D1C1D0C1CFC1CEC1CDC1CCC1CBC18E
:10001000CAC1C9C117C30EC4C6C1C5C1C4C1C3C109
:10002000C2C1C1C137C7BFC1ADC8BDC1BCC1BBC161
:10003000BAC1B9C163C665C668C66AC66CC66EC6B3
:1000400070C672C674C676C678C67AC60C52657318
:10005000657420312E3730000A0D6E6F2077696E7F
:10006000642020203D200009392E3020202D202022
:10007000392E39203D20000D312E30202D20312EFB
:1000800039203D20000931302E30202D2031302EF6
:1000900039203D20000D322E30202D20322E3920E7
:1000A0003D20000931312E30202D2031312E3920D4
:1000B0003D20000D332E30202D20332E39203D20C1
:1000C000000931322E30202D2031322E39203D20B2
:1000D000000D342E30202D20342E39203D200009F3
:1000E00031332E30202D2031332E39203D20000D8C
:1000F000352E30202D20352E39203D200009313479
:100100002E30202D2031342E39203D20000D362E6A
:1001100030202D20362E39203D20000931352E305B
:10012000202D2031352E39203D20000D372E302056
:100130002D20372E39203D20000931362E30202D3C
:100140002031362E39203D20000D382E30202D2034
:10015000382E39203D20000931372E3020262055F9
:10016000702020203D20000A0D45726173652061DA
:100170006C6C206C6F676765642064617461202813
:10018000792F6E29000A0D446F6E65004A616E007A
:10019000466562004D617200417072004D617900E8
:1001A0004A756E004A756C004175670053657000B2
:1001B0004F6374004E6F7600446563000A0D5573FB
:1001C00065204152524F57204B65797320746F2040
:1001D00073656C656374206D6F6E74680D000D56E9
:1001E0006261747409093D20000C47657420446104
:1001F000746120666F72207768696368204D6F6E46
:1002000074683F000A0A0D4D6F6E74682773204DA5
:100210006178696D756D207370656564203D20009F
:100220000C536574204D6F6E7468000C6D203D207A
:10023000000A0D456E74657220536C6F7065200066
:100240000D6D203D20000C62203D20000A0D456E02
:10025000746572204F666673657420000D62203DE0
:1002600020000C43616C6962726174696F6E204D8D
:100270006F6465204F4E000C43616C69627261745B
:10028000696F6E204D6F6465204F4646000C4669CD
:10029000726D77617265093D20312E3730000D4C4B
:1002A0006F6767696E67204D6F6E7468093D200047
:1002B0000D44617973206C6F67676564093D2000A8
:1002C0000D23206F6620726573657473093D2000ED
:1002D0000D43757272656E74207370656564093DB7
:1002E00020000D4F666673657420286229093D2041
:1002F000000D536C6F706520286D29093D20000C9E
:100300005072657373200D205B675D6574206461B6
:1003100074610D205B635D6C656172206461746162
:100320000D205B735D6574206D6F6E74680D205BCE
:10033000695D6E666F000D205B6D5D20736C6F7084
:10034000650D205B625D206F66667365740D205BD2
:10035000745D6F67676C652063616C69627261745C
:10036000696F6E206D6F64650D205B725D657365EE
:10037000740011241FBECFEFD4E0DEBFCDBF11E06B
:10038000A0E0B1E0EEE7F2E102C005900D92A030EE
:10039000B107D9F711E0A0E0B1E001C01D92AC3F78
:1003A000B107E1F74FC02CCEF999FECF92BD81BDC8
:1003B000F89A80B599270895F999FECF92BD81BD2D
:1003C00060BDF89484E08FBBF99A78940895282F43
:1003D00091E0F8948091FA0187FF90E07894992356
:1003E000C1F7F8948091F701882331F42093C60077
:1003F00081E08093F70111C080910001E82FFF2771
:10040000EF77F070E85AFE4F20838F5F80930001F2
:100410008091FA018F5F8093FA0178940895CF93C9
:10042000DF93EC01A895FC018491882341F0FE0143
:100430008491CDDF2196FE0184918823C1F7DF915D
:10044000CF910895CFEFD4E0DEBFCDBFF89488E11F
:10045000809360008FE08093600021E025B982E006
:1004600087B984B9299889E18093C4001092C000AB
:1004700088ED8093C100109280008DE08093810010
:100480008FE99FE0909389008093880082E28093B7
:100490006F0023BF85EE80936400789410920D0165
:1004A00083E090E081DF809333018093DB01992723
:1004B00047967ADF8093E0018CE490E0B0DF909182
:1004C000330184E2989FC00111249093DA01809354
:1004D000D90110920B0180910B01082F1127000FF9
:1004E000111F025F1E4FF801118210828091D90105
:1004F0009091DA0159DF9927382F2227F80180815E
:100500009181822B932B9183808380910B01082F03
:100510001127000F111F025F1E4F8091D90190918A
:10052000DA01019641DF282F3327F801808191817C
:10053000822B932B9183808340910B01E42FFF2723
:10054000EE0FFF1FE25FFE4F8091DE019091DF0111
:1005500020813181820F931F9093DF018093DE0110
:100560008091D9019091DA0102969093DA018093FB
:10057000D901842F8F5F80930B01823108F4ABCFB8
:1005800080E090E011DF9927182F002781E090E0AC
:100590000BDF9927082B192B1093F9010093F80111
:1005A00082E090E001DF80930A0184E090E0FCDECD
:1005B00080930C018A3F38F48F5F80930C01682F81
:1005C00084E090E0F9DE8895FECFEF92FF920F93E2
:1005D0001F938C0170E1E72E77E2F72EB701FED56D
:1005E000CB01805DF4DEC801B701F8D58C0168EE5F
:1005F000E62E63E0F62EB701F1D5CB01805DE7DE94
:10060000C801B701EBD58C0154E6E52EF12CB701FA
:10061000E5D5CB01805DDBDEC801B701DFD58C01FC
:100620004AE0E42EF12CB701D9D5CB01805DCFDEB5
:10063000C801B701D3D5805DCADE1F910F91FF902D
:10064000EF9008951F920F920FB60F921124EF9220
:10065000FF920F931F932F933F934F935F936F934B
:100660007F938F939F93AF93BF93EF93FF934091AB
:100670008600509187008091FB01843010F0109229
:10068000FB012091F3013091F40142175307E8F484
:10069000B09B1BC08091FB01E82FFF27EE0FFF1FCF
:1006A000EE5FFE4F8091DC019091DD01840F951F7C
:1006B000821B930B8056904F9183808380E690EF4E
:1006C0009093DD018093DC0116C08091FB01E82F3F
:1006D000FF27EE0FFF1FEE5FFE4F8091DC01909130
:1006E000DD01840F951F821B930B918380831092F1
:1006F000DD011092DC015093F4014093F3018091ED
:10070000FB018F5F8093FB018091F8019091F901CB
:100710007C010027112780910201909103019C0127
:10072000442755278091040190910501AA27BB27F2
:10073000280F391F4A1F5B1F809106019091070106
:10074000AA27BB27280F391F4A1F5B1F809108016A
:1007500090910901AA27BB27280F391F4A1F5B1F49
:10076000F2E05595479537952795FA95D1F7C80149
:10077000B70148D5DA01C90120910A01280F209359
:10078000D8019091D8018091E001891760F480919F
:10079000D8018093E00190913301292F3327682FEE
:1007A000C901479609DE80910D01882371F18DE022
:1007B0000EDE8091020190910301AA27BB272091B0
:1007C00004013091050144275527820F931FA41F70
:1007D000B51F209106013091070144275527820F4C
:1007E000931FA41FB51F20910801309109014427D0
:1007F0005527820F931FA41FB51FE2E0B595A7955B
:1008000097958795EA95D1F7E0DEFF91EF91BF913B
:10081000AF919F918F917F916F915F914F913F9198
:100820002F911F910F91FF90EF900F900FBE0F909F
:100830001F9018951F920F920FB60F9211242F93AD
:100840003F934F935F936F937F938F939F93AF9358
:10085000BF93EF93FF934091DC015091DD019A012A
:1008600024523A4F8091F8019091F90128173907E5
:1008700038F44056504F5093DD014093DC0102C0E4
:100880001092D801A8958091D801823118F081E1A9
:100890008093D8018091D801E82FFF27EF51FE4FB8
:1008A00080818B3350F48091D801E82FFF27EF51DE
:1008B000FE4F80818F5F808314C08091D801E82F24
:1008C000FF27EE0FFF1FE25FFE4F808191810196AF
:1008D000918380838091D801E82FFF27EF51FE4F4D
:1008E0001082809132018B3320F48F5F809332012C
:1008F0006EC0109232018091DE019091DF0101966D
:100900009093DF018093DE0188519B4A08F45FC019
:100910001092DF011092DE019091330184E2989FE2
:10092000C00111249093DA018093D90110920B0138
:1009300080910B01E82FFF27EE0FFF1FE25FFE4FB4
:1009400080819181892F9927682F8091D901909179
:10095000DA0132DD80910B01E82FFF27EE0FFF1F38
:10096000E25FFE4F8091D9019091DA01608101969A
:1009700023DD8091D9019091DA0102969093DA01FA
:100980008093D90180910B01E82FFF27EE0FFF1F05
:10099000E25FFE4F118210828F5F80930B018231E4
:1009A00038F2809133018C3010F48F5F01C081E008
:1009B000809333016091330183E090E0FDDC10927D
:1009C000E00180913301992760E04796F5DC809142
:1009D000F5019091F60101969093F6018093F5014F
:1009E00080539A4208F441C01092F6011092F5012A
:1009F0009091330184E2989FC00111249093DA0111
:100A00008093D90110920B0180910B01E82FFF27F1
:100A1000EE0FFF1FE25FFE4F80819181892F9927A2
:100A2000682F8091D9019091DA01C6DC80910B0189
:100A3000E82FFF27EE0FFF1FE25FFE4F8091D901E5
:100A40009091DA0160810196B7DC8091D901909193
:100A5000DA0102969093DA018093D90180910B011B
:100A60008F5F80930B01823178F2FF91EF91BF91FC
:100A7000AF919F918F917F916F915F914F913F9136
:100A80002F910F900FBE0F901F9018950F931F93EB
:100A90008C0188E590E0C3DCF8018081918195DDCF
:100AA00087E690E0BCDCF801828993898EDD87E7D8
:100AB00090E0B5DCF8018281938187DD85E890E0E4
:100AC000AEDCF8018489958980DD85E990E0A7DCBA
:100AD000F8018481958179DD83EA90E0A0DCF8015A
:100AE0008689978972DD83EB90E099DCF801868135
:100AF00097816BDD81EC90E092DCF801808D918D27
:100B000064DD81ED90E08BDCF801808591855DDD11
:100B10008FED90E084DCF801828D938D56DD8FEEB1
:100B200090E07DDCF801828593854FDD8DEF90E0CC
:100B300076DCF801848D958D48DD8DE091E06FDCE9
:100B4000F8018485958541DD8BE191E068DCF80151
:100B5000868D978D3ADD8BE291E061DCF801868528
:100B6000978533DD89E391E05ADCF80180A191A1FA
:100B70002CDD89E491E053DCF8018089918925DD41
:100B800087E591E04CDCF80182A193A11EDD1F9165
:100B90000F910895DF92EF92FF920F931F93CF93DF
:100BA000DF93CDB7DEB725970FB6F894DEBF0FBE43
:100BB000CDBF8091C1008F778093C100EE24FF24C8
:100BC00000E0D02E09830A830B830C830D83809170
:100BD000C00087FD02C0A895FACF1091C6001D3055
:100BE000C9F40023A9F19E012F5F3F4FC70113E015
:100BF000880F991F1A95E1F78E0D9F1DE80EF91EBB
:100C0000F901ED0DF11D8081E80EF11CD394015026
:100C100069F71EC0183061F40023C9F20150FE01CB
:100C2000E00FF11D1182812FD2DB80E2D0DB0DC0FD
:100C3000053068F6103358F21A3348F6FE01E00F1B
:100C4000F11D10531183105D0F5F812FC0DBBFCFEB
:100C50008091C10080688093C100C70125960FB6BE
:100C6000F894DEBF0FBECDBFDF91CF911F910F91E2
:100C7000FF90EF90DF9008958091C1008F7780936F
:100C8000C10087E691E0CBDB8091C00087FD02C008
:100C9000A895FACF8091C6008937E1F488E190E009
:100CA0009093DA018093D90160E08091D90190910D
:100CB000DA0182DB8091D9019091DA01019690935B
:100CC000DA018093D901845D914070F361E083E0A3
:100CD00090E072DB8091C10080688093C10085E85C
:100CE00091E09DDB08959927AA27BB27FC01319746
:100CF000EC30F10540F5E65EFF4F09948CE891E099
:100D000002C080E991E08BDB089584E991E0FBCF9C
:100D100088E991E0F8CF8CE991E0F5CF80EA91E0A5
:100D2000F2CF84EA91E0EFCF88EA91E0ECCF8CEA51
:100D300091E0E9CF80EB91E0E6CF84EB91E0E3CF67
:100D400088EB91E06CDB0895CF938091C1008F77A1
:100D50008093C100809133018093DB01C5E48CEB6B
:100D600091E05DDBC154C53048F48091DB01BBDF0D
:100D700088E02DDB88E02BDB88E029DB8091C00058
:100D800087FD02C0A895FACFC091C600CD3031F4DE
:100D90008091C10080688093C1001BC08C2F825459
:100DA000823048F48091DB018C3010F48F5F01C0F9
:100DB00081E08093DB01C13411F0C43499F6809155
:100DC000DB01823010F0815001C08CE08093DB01A8
:100DD000C9CFCF9108950F931F93809164008E7FA8
:100DE00080936400419A80E480937C0087EE809336
:100DF0007A0080917A0084FFFCCF80917A00806134
:100E000080937A0080917A0084FFFCCF0091780073
:100E100010917900000F111F809178009091790056
:100E200096958795080F191F419810927A00809126
:100E300064008160809364008EED91E0F0DAC80177
:100E400068EE73E0CBD1CB01805DC1DAC80168EEFA
:100E500073E0C4D18C0164E670E0C0D1CB01805D49
:100E6000B6DAC80164E670E0B9D18C018EE2AFDA7F
:100E7000C8016AE070E0B2D1CB01805DA8DAC80198
:100E80006AE070E0ABD1805DA2DA86E7A0DA1F915C
:100E90000F9108951F920F920FB60F9211240F9386
:100EA0001F932F933F934F935F936F937F938F93F2
:100EB0009F93AF93BF93EF93FF938091C6008736C4
:100EC00009F067C089EE91E0AADA3EDF9091DB017C
:100ED00080913301981709F44FC084E2989FC001B4
:100EE00011249093DA018093D90110920B01809123
:100EF0000B01082F1127000F111F0C5C1E4FF8016A
:100F0000118210828091D9019091DA014DDA9927EE
:100F1000382F2227F80180819181822B932B918396
:100F2000808380910B01082F1127000F111F0C5C8B
:100F30001E4F8091D9019091DA01019635DA282F60
:100F40003327F80180819181822B932B91838083B9
:100F50008091D9019091DA0102969093DA01809301
:100F6000D90180910B018F5F80930B01823108F4CE
:100F7000BECF84E391E002C08EE091E087DD84E0A3
:100F800092E04DDA8091DB01992747960DDA992797
:100F9000DEC0833709F050C080E292E040DAD4DE50
:100FA0008091DB0180933301682F83E090E004DAC5
:100FB0001092E00180913301992760E04796FCD9B7
:100FC0001092DF011092DE019091330184E2989F2C
:100FD000C00111249093DA018093D90110920B0182
:100FE00060E08091D9019091DA01E6D98091D90130
:100FF0009091DA0160E00196DFD98091D90190915A
:10100000DA0102969093DA018093D90180910B0165
:10101000E82FFF27EE0FFF1FE25FFE4F11821082C5
:101020008F5F80930B018231D8F210920C0160E047
:1010300084E090E0C1D993C08D36F1F48BE292E068
:10104000EED98091F8019091F901BFDA81E392E045
:10105000E6D9A0DD9093F9018093F801892F9927B3
:10106000682F80E090E0A8D96091F80181E090E0DD
:10107000A3D980E492E066C08236B9F486E492E0B7
:10108000CED980910A019927A0DA8CE492E0C7D9E1
:1010900081DD80930A01682F82E090E08DD98CE594
:1010A00092E0BDD980910A0172CF843779F48091A2
:1010B0000D01882331F481E080930D0182E692E0F6
:1010C0004DC010920D0187E792E048C0833611F4BD
:1010D000D3DD45C0823739F488E18093600088E031
:1010E00080936000FFCF8936A1F58DE892E097D913
:1010F0008EE992E094D980913301F5DD80EB92E0A6
:101100008ED98091DE019091DF0160EA75E066D0B2
:10111000CB015BDA80EC92E082D980910C019927B7
:1011200054DA80ED92E07BD98091D80199274DDA8D
:1011300052DE82EE92E073D980910A01992745DA56
:1011400081EF92E06CD98091F8019091F9013DDA3C
:1011500006C08FEF92E063D986E393E060D9FF91F8
:10116000EF91BF91AF919F918F917F916F915F911F
:101170004F913F912F911F910F910F900FBE0F90A4
:101180001F9018951F920F920FB60F9211248F93F4
:101190009F93EF93FF938091FA018823A1F09091A0
:1011A0000101E92FFF27EF77F070E85AFE4F8081A9
:1011B0008093C6009F5F909301018091FA01815056
:1011C0008093FA0102C08093F701FF91EF919F9104
:1011D0008F910F900FBE0F901F901895AA1BBB1BED
:1011E00051E107C0AA1FBB1FA617B70710F0A61B27
:1011F000B70B881F991F5A95A9F780959095BC0148
:10120000CD01089597FB092E05260ED057FD04D079
:1012100014D00AD0001C38F4509540953095219593
:101220003F4F4F4F5F4F0895F6F79095809570951B
:1012300061957F4F8F4F9F4F0895A1E21A2EAA1BF1
:10124000BB1BFD010DC0AA1FBB1FEE1FFF1FA21776
:10125000B307E407F50720F0A21BB30BE40BF50B73
:10126000661F771F881F991F1A9469F760957095FC
:0E127000809590959B01AC01BD01CF010895C2
:00000001FF
